******************************************************************************
                  TI ARM Linker PC v5.0.4                      
******************************************************************************
>> Linked Fri Jun 22 09:26:24 2018

OUTPUT FILE NAME:   <TMS570LS07x_MCAL.out>
ENTRY POINT SYMBOL: "_c_int00"  address: 00010854


MEMORY CONFIGURATION

         name            origin    length      used     unused   attr    fill
----------------------  --------  ---------  --------  --------  ----  --------
  VECTORS               00000000   00000020  00000020  00000000     X
  FLASH0                00000020   000bffe0  00012cf2  000ad2ee  R  X
  STACKS                08000000   00001500  00000000  00001500  RW  
  RAM                   08001500   0001eb00  00000aaa  0001e056  RW  


SEGMENT ALLOCATION MAP

run origin  load origin   length   init length attrs members
----------  ----------- ---------- ----------- ----- -------
00000000    00000000    00012d18   00012d18    r-x
  00000000    00000000    00000020   00000020    r-x .intvecs
  00000020    00000020    000114f8   000114f8    r-x .text
  00011518    00011518    00000cd8   00000cd8    r-x FEE_TEXT_SECTION
  000121f0    000121f0    00000756   00000756    r-- .const
  00012948    00012948    0000028c   0000028c    r-- FEE_CONST_SECTION
  00012bd8    00012bd8    00000140   00000140    r-- .cinit
08001500    08001500    00000aad   0000097d    rw-
  08001500    08001500    00000844   00000844    rw- .data
  08001d44    08001d44    00000139   00000139    rw- FEE_DATA_SECTION
  08001e80    08001e80    0000012d   00000000    rw- .bss


SECTION ALLOCATION MAP

 output                                  attributes/
section   page    origin      length       input sections
--------  ----  ----------  ----------   ----------------
.intvecs   0    00000000    00000020     
                  00000000    00000020     sys_intvecs.obj (.intvecs)

.text      0    00000020    000114f8     
                  00000020    000025f8     ti_fee_util.obj (.text)
                  00002618    00001e94     Can.obj (.text)
                  000044ac    000014d0     Spi_Dlc.obj (.text)
                  0000597c    00001214     Adc.obj (.text)
                  00006b90    00001014     Icu.obj (.text)
                  00007ba4    00000e98     Port_PBcfg.obj (.text)
                  00008a3c    00000d30     Gpt.obj (.text)
                  0000976c    00000c80     Pwm.obj (.text)
                  0000a3ec    00000a48     Spi_Hw.obj (.text)
                  0000ae34    00000990     ti_fee_ini.obj (.text)
                  0000b7c4    00000980     Lin.obj (.text)
                  0000c144    000006e0     Mcu.obj (.text)
                  0000c824    0000067c     ti_fee_main.obj (.text)
                  0000cea0    00000630     sys_vim.obj (.text)
                  0000d4d0    00000568     system.obj (.text)
                  0000da38    000004c8     Dio.obj (.text)
                  0000df00    000004b4     Fee.obj (.text)
                  0000e3b4    00000400     pinmux.obj (.text)
                  0000e7b4    000003b8     sci.obj (.text)
                  0000eb6c    0000034c     sys_core.obj (.text)
                  0000eeb8    00000324     esm.obj (.text)
                  0000f1dc    00000304     main.obj (.text)
                  0000f4e0    00000290     Spi_Irq.obj (.text:retain)
                  0000f770    00000260     F021_API_CortexR4_BE_V3D16.lib : FlashStateMachine.InitializeFlashBanks.obj (.text:Fapi_initializeFlashBanks)
                  0000f9d0    0000020c     Spi_DlcDma.obj (.text)
                  0000fbdc    00000200     Wdg.obj (.text)
                  0000fddc    000001b8     Port.obj (.text)
                  0000ff94    00000180     Adc_Irq.obj (.text:retain)
                  00010114    0000017c     F021_API_CortexR4_BE_V3D16.lib : FlashStateMachine.SetActiveBank.obj (.text:Fapi_setActiveFlashBank)
                  00010290    00000158     sys_vim.obj (.text:retain)
                  000103e8    00000154     sci.obj (.text:retain)
                  0001053c    00000130     Pwm_Het.obj (.text)
                  0001066c    00000124     Icu_Het.obj (.text)
                  00010790    000000c4     esm.obj (.text:retain)
                  00010854    000000c0     sys_startup.obj (.text:retain)
                  00010914    000000ae     rtsv7R4_T_be_v3D16_eabi.lib : floor.obj (.text)
                  000109c2    00000002     --HOLE-- [fill = 0]
                  000109c4    000000a8     Can_Irq.obj (.text:retain)
                  00010a6c    000000a4     Gpt_Irq.obj (.text:retain)
                  00010b10    0000009c     Can_misc.obj (.text)
                  00010bac    0000009c     rtsv7R4_T_be_v3D16_eabi.lib : memcpy_t2.obj (.text)
                  00010c48    00000098                                 : auto_init.obj (.text)
                  00010ce0    00000094     F021_API_CortexR4_BE_V3D16.lib : BlankCheck.obj (.text:Fapi_doBlankCheck)
                  00010d74    00000080                                    : FlashStateMachine.EnableEepromSectors.obj (.text:Fapi_enableEepromBankSectors)
                  00010df4    00000070     Pwm_Irq.obj (.text:retain)
                  00010e64    00000060     rtsv7R4_T_be_v3D16_eabi.lib : copy_decompress_rle.obj (.text)
                  00010ec4    0000005e     F021_API_CortexR4_BE_V3D16.lib : Read.LoopDword.obj (.text:_Fapi_loopRegionForValue)
                  00010f22    00000002     --HOLE-- [fill = 0]
                  00010f24    00000054     rtsv7R4_T_be_v3D16_eabi.lib : u_div32.obj (.text)
                  00010f78    00000050     F021_API_CortexR4_BE_V3D16.lib : FlashStateMachine.Hercules.IsEccAddress.obj (.text:Fapi_isAddressEcc)
                  00010fc8    00000048     rtsv7R4_T_be_v3D16_eabi.lib : cpy_tbl.obj (.text)
                  00011010    00000044     F021_API_CortexR4_BE_V3D16.lib : FlashStateMachine.EnableEepromSectors.obj (.text:_Fapi_EnableSectors)
                  00011054    00000040     det.obj (.text)
                  00011094    00000040     rtsv7R4_T_be_v3D16_eabi.lib : exit.obj (.text)
                  000110d4    0000003c     F021_API_CortexR4_BE_V3D16.lib : FlashStateMachine.IssueFsmCommand.obj (.text:_Fapi_issueFsmCommand)
                  00011110    0000003c     Lin_Irq.obj (.text:retain)
                  0001114c    00000038     Icu_Irq.obj (.text:retain)
                  00011184    00000038     Wdg_Irq.obj (.text:retain)
                  000111bc    00000036     F021_API_CortexR4_BE_V3D16.lib : Utilities.CalculateFletcher.obj (.text:Fapi_calculateFletcherChecksum)
                  000111f2    00000002     --HOLE-- [fill = 0]
                  000111f4    00000030                                    : Async.WithAddress.obj (.text:Fapi_issueAsyncCommandWithAddress)
                  00011224    00000030                                    : Utilities.WaitDelay.obj (.text:Fapi_waitDelay)
                  00011254    0000002c                                    : Read.Common.obj (.text:_Fapi_readDword)
                  00011280    0000002a                                    : Async.obj (.text:Fapi_issueAsyncCommand)
                  000112aa    00000002     --HOLE-- [fill = 0]
                  000112ac    00000028     SchM_Mcu.obj (.text)
                  000112d4    00000028     sys_startup.obj (.text)
                  000112fc    00000024     SchM_Pwm.obj (.text)
                  00011320    00000022     F021_API_CortexR4_BE_V3D16.lib : Read.FlushPipeline.obj (.text:Fapi_flushPipeline)
                  00011342    00000002     --HOLE-- [fill = 0]
                  00011344    00000020     SchM_Adc.obj (.text)
                  00011364    00000020     SchM_Can.obj (.text)
                  00011384    00000020     SchM_Dio.obj (.text)
                  000113a4    00000020     SchM_Gpt.obj (.text)
                  000113c4    00000020     SchM_Icu.obj (.text)
                  000113e4    00000020     SchM_Port.obj (.text)
                  00011404    00000020     SchM_Spi.obj (.text)
                  00011424    0000001c     F021_API_CortexR4_BE_V3D16.lib : FlashStateMachine.InitializeFlashBanks.obj (.text:_Fapi_divideUnsignedLong)
                  00011440    00000018     notification.obj (.text)
                  00011458    00000014     rtsv7R4_T_be_v3D16_eabi.lib : _lock.obj (.text)
                  0001146c    00000014                                 : icall16.obj (.text)
                  00011480    00000012                                 : copy_zero_init.obj (.text:decompress:ZI)
                  00011492    00000002     --HOLE-- [fill = 0]
                  00011494    00000010     F021_API_CortexR4_BE_V3D16.lib : Utilities.GetNumberOfSectors.obj (.text:Fapi_getNumberOfBankSectors)
                  000114a4    00000010                                    : FlashStateMachine.ScaleFclk.obj (.text:_scaleEEFclk)
                  000114b4    00000010                                    : FlashStateMachine.ScaleFclk.obj (.text:_scaleMainFclk)
                  000114c4    0000000e     rtsv7R4_T_be_v3D16_eabi.lib : copy_decompress_none.obj (.text:decompress:none)
                  000114d2    0000000c     F021_API_CortexR4_BE_V3D16.lib : Read.WdService.obj (.text:_Fapi_checkWdService)
                  000114de    00000002     --HOLE-- [fill = 0]
                  000114e0    00000008     EcuM_Cbk.obj (.text)
                  000114e8    00000008     Fapi_UserDefinedFunctions.obj (.text)
                  000114f0    00000006     rtsv7R4_T_be_v3D16_eabi.lib : copy_decompress_rle.obj (.text:decompress:rle24)
                  000114f6    00000002     --HOLE-- [fill = 0]
                  000114f8    00000004     dem.obj (.text)
                  000114fc    00000004     sys_phantom.obj (.text:retain)
                  00011500    0000000a     Fapi_UserDefinedFunctions.obj (.tramp.Fapi_serviceWatchdogTimer.1)
                  0001150a    00000002     --HOLE-- [fill = 0]
                  0001150c    0000000c     F021_API_CortexR4_BE_V3D16.lib : FlashStateMachine.EnableEepromSectors.obj (.tramp.Fapi_enableEepromBankSectors.1)

FEE_TEXT_SECTION 
*          0    00011518    00000cd8     
                  00011518    000004d4     ti_fee_writeAsync.obj (FEE_TEXT_SECTION)
                  000119ec    0000039c     ti_fee_read.obj (FEE_TEXT_SECTION)
                  00011d88    00000204     ti_fee_eraseimmediateblock.obj (FEE_TEXT_SECTION)
                  00011f8c    000001c8     ti_fee_invalidateblock.obj (FEE_TEXT_SECTION)
                  00012154    0000009c     ti_fee_cancel.obj (FEE_TEXT_SECTION)

.const     0    000121f0    00000756     
                  000121f0    00000200     sys_vim.obj (.const:s_vim_init)
                  000123f0    000000c4     Pwm_PBcfg.obj (.const)
                  000124b4    000000c0     Adc_PBcfg.obj (.const:Adc_GroupConfigList0_at)
                  00012574    000000b4     Port_PBcfg.obj (.const:Port_RefreshConfig0_at)
                  00012628    00000094     Spi_PBcfg.obj (.const)
                  000126bc    0000007c     Icu_PBcfg.obj (.const)
                  00012738    00000058     Mcu_PBcfg.obj (.const)
                  00012790    00000040     Gpt_PBcfg.obj (.const:Gpt_ChannelConfig0)
                  000127d0    00000030     Port_PBcfg.obj (.const)
                  00012800    0000002c     Adc_PBcfg.obj (.const)
                  0001282c    00000028     Dio_PBcfg.obj (.const)
                  00012854    00000028     Pwm_PBcfg.obj (.const:Pwm_Het1Program_Cfg0)
                  0001287c    00000028     Pwm_PBcfg.obj (.const:Pwm_Het2Program_Cfg0)
                  000128a4    00000024     Mcu_PBcfg.obj (.const:Mcu_Sys1RegConfiguration)
                  000128c8    00000020     Can.obj (.const)
                  000128e8    00000010     Can_PBcfg.obj (.const)
                  000128f8    00000010     Gpt.obj (.const)
                  00012908    0000000c     Icu.obj (.const)
                  00012914    0000000a     Spi_Dlc.obj (.const)
                  0001291e    00000002     --HOLE-- [fill = 0]
                  00012920    0000000a     Spi_DlcDma.obj (.const)
                  0001292a    00000002     --HOLE-- [fill = 0]
                  0001292c    00000008     main.obj (.const:.string)
                  00012934    00000008     Gpt_PBcfg.obj (.const)
                  0001293c    00000004     Spi_Dlc.obj (.const:.string)
                  00012940    00000003     Icu.obj (.const:.string)
                  00012943    00000001     --HOLE-- [fill = 0]
                  00012944    00000002     Spi_PBcfg.obj (.const:.string)

FEE_CONST_SECTION 
*          0    00012948    0000028c     
                  00012948    000001a4     Device_TMS570LS07.obj (FEE_CONST_SECTION)
                  00012aec    000000e8     fee_cfg.obj (FEE_CONST_SECTION)

.cinit     0    00012bd8    00000140     
                  00012bd8    00000103     (.cinit..data.load) [load image, compression = rle]
                  00012cdb    00000001     --HOLE-- [fill = 0]
                  00012cdc    0000000c     (__TI_handler_table)
                  00012ce8    0000000b     (.cinit.FEE_DATA_SECTION.load) [load image, compression = rle]
                  00012cf3    00000005     --HOLE-- [fill = 0]
                  00012cf8    00000008     (.cinit..bss.load) [load image, compression = zero_init]
                  00012d00    00000018     (__TI_cinit_table)

.data      0    08001500    00000844     
                  08001500    00000358     Can.obj (.data)
                  08001858    00000114     main.obj (.data)
                  0800196c    00000110     Icu.obj (.data)
                  08001a7c    000000ec     Spi_Dlc.obj (.data)
                  08001b68    000000e8     Can_PBcfg.obj (.data)
                  08001c50    00000038     Spi_PBcfg.obj (.data)
                  08001c88    0000002c     Gpt.obj (.data)
                  08001cb4    00000028     Pwm.obj (.data)
                  08001cdc    00000018     Lin.obj (.data)
                  08001cf4    0000000c     Adc.obj (.data)
                  08001d00    0000000c     Wdg.obj (.data)
                  08001d0c    00000008     Can_misc.obj (.data)
                  08001d14    00000008     F021_API_CortexR4_BE_V3D16.lib : FlashStateMachine.ScaleFclk.obj (.data)
                  08001d1c    00000008     Spi_DlcDma.obj (.data)
                  08001d24    00000008     rtsv7R4_T_be_v3D16_eabi.lib : _lock.obj (.data)
                  08001d2c    00000008                                 : exit.obj (.data)
                  08001d34    00000005     Spi.obj (.data)
                  08001d39    00000001     F021_API_CortexR4_BE_V3D16.lib : FlashStateMachine.SetActiveBank.obj (.data)
                  08001d3a    00000002     --HOLE--
                  08001d3c    00000004     Mcu.obj (.data)
                  08001d40    00000004     Port.obj (.data)

FEE_DATA_SECTION 
*          0    08001d44    00000139     
                  08001d44    00000118     ti_fee_ini.obj (FEE_DATA_SECTION) [fill = 0]
                  08001e5c    00000020     ti_fee_util.obj (FEE_DATA_SECTION:init)
                  08001e7c    00000001     ti_fee_main.obj (FEE_DATA_SECTION)

.bss       0    08001e80    0000012d     UNINITIALIZED
                  08001e80    000000c8     Spi_Hw.obj (.bss)
                  08001f48    00000028     sci.obj (.bss:g_sciTransfer_t)
                  08001f70    00000024     Adc_PBcfg.obj (.bss:Adc_GroupDataListRt0Hw1_at)
                  08001f94    0000000c     Adc_PBcfg.obj (.bss)
                  08001fa0    00000008     det.obj (.bss)
                  08001fa8    00000004     Can.obj (.bss)
                  08001fac    00000001     Can_misc.obj (.bss)


LINKER GENERATED COPY TABLES

__TI_cinit_table @ 00012d00 records: 3, size/record: 8, table size: 24
	.data: load addr=00012bd8, load size=00000103 bytes, run addr=08001500, run size=00000844 bytes, compression=rle
	FEE_DATA_SECTION: load addr=00012ce8, load size=0000000b bytes, run addr=08001d44, run size=00000139 bytes, compression=rle
	.bss: load addr=00012cf8, load size=00000008 bytes, run addr=08001e80, run size=0000012d bytes, compression=zero_init


LINKER GENERATED HANDLER TABLE

__TI_handler_table @ 00012cdc records: 3, size/record: 4, table size: 12
	index: 0, handler: __TI_zero_init
	index: 1, handler: __TI_decompress_rle24
	index: 2, handler: __TI_decompress_none

VENEERS

callee name               veneer name
   callee addr  veneer addr  call addr  call info
--------------  -----------  ---------  ----------------
Fapi_serviceWatchdogTimer  $Ven$TA$L$PI$$Fapi_serviceWatchdogTimer
   000114e8     00011500     000114d8   F021_API_CortexR4_BE_V3D16.lib : Read.WdService.obj (.text:_Fapi_checkWdService)
Fapi_enableEepromBankSectors  $Ven$AT$L$PI$$Fapi_enableEepromBankSectors
   00010d75     0001150c     000001ec   ti_fee_util.obj (.text)

[2 trampolines]
[2 trampoline calls]


GLOBAL SYMBOLS: SORTED ALPHABETICALLY BY Name 

address    name
--------   ----
00012820   AdcConfigSet_0
00006b88   Adc_AvoidNotification
00006998   Adc_DeInit
000068d8   Adc_DisableGroupNotification
000067a0   Adc_EnableGroupNotification
00006664   Adc_GetGroupStatus
00006474   Adc_GetStreamLastPointer
00006428   Adc_GetVersionInfo
00012800   Adc_HwUnitConfigList0_at
0000627c   Adc_Init
00006214   Adc_IrqFunction
000100d4   Adc_IsrUnit0Ev
00010094   Adc_IsrUnit0G1
00010054   Adc_IsrUnit0G2
00010014   Adc_IsrUnit1Ev
0000ffd4   Adc_IsrUnit1G1
0000ff94   Adc_IsrUnit1G2
00006160   Adc_ProcessBufferCircular
000060ac   Adc_ProcessBufferLinear
0000603c   Adc_ProcessBufferSingle
00006000   Adc_ProcessConversionCircular
00005fa0   Adc_ProcessConversionLinear
00005f74   Adc_ProcessConversionSingle
00005d84   Adc_ReadGroup
00005d18   Adc_SetupResultBuffer
00005a70   Adc_StartGroupConversion
0000597c   Adc_StopGroupConversion
0800187c   Adc_result_buffer
00011095   C$$EXIT
08001860   CAN_RX_Done_Flag
0800185c   CAN_RX_Int_Flag
08001864   CAN_TX_Done_Flag
08001506   CanBusOffRecoveryStatus
000128e8   CanConfigSet_0
08001bac   CanConfigSet_0_CanController_0
08001ba0   CanConfigSet_0_CanController_0_BaudRateConfigList
08001b80   CanConfigSet_0_CanController_0_CanControllerBaudrateConfig_0
08001b68   CanConfigSet_0_CanController_0_CanFilterMask_0
08001b74   CanConfigSet_0_CanController_0_FilterMaskList
08001bcc   CanConfigSet_0_CanController_1
08001ba4   CanConfigSet_0_CanController_1_BaudRateConfigList
08001b8a   CanConfigSet_0_CanController_1_CanControllerBaudrateConfig_0
08001b6c   CanConfigSet_0_CanController_1_CanFilterMask_0
08001b78   CanConfigSet_0_CanController_1_FilterMaskList
08001bec   CanConfigSet_0_CanController_2
08001ba8   CanConfigSet_0_CanController_2_BaudRateConfigList
08001b94   CanConfigSet_0_CanController_2_CanControllerBaudrateConfig_0
08001b70   CanConfigSet_0_CanController_2_CanFilterMask_0
08001b7c   CanConfigSet_0_CanController_2_FilterMaskList
08001c0c   CanConfigSet_0_CanController_List
08001c18   CanConfigSet_0_CanHardwareObject_0
08001c30   CanConfigSet_0_CanHardwareObject_1
08001c48   CanConfigSet_0_CanHardwareObject_List
080016d8   CanHtrhMbMapping
00010b80   CanIf_ControllerBusOff
00010b68   CanIf_ControllerModeIndication
00010b34   CanIf_RxIndication
00010b10   CanIf_TxConfirmation
08001558   CanMbMapping
08001868   CanRxData
0800151a   CanSduPtr
00010a34   Can_0_Int0ISR
00004354   Can_0_Int0ISR_Fun
000109fc   Can_1_Int0ISR
0000422c   Can_1_Int0ISR_Fun
000109c4   Can_2_Int0ISR
00004100   Can_2_Int0ISR_Fun
0800153c   Can_CanConfig
00003e2c   Can_ChangeBaudrate
00003d10   Can_CheckBaudrate
00003c54   Can_CheckWakeup
00003b7c   Can_ConfigRegReadBack
00003ad0   Can_DisableControllerInterrupts
000039d4   Can_EnableControllerInterrupts
00003910   Can_GetVersionInfo
0000384c   Can_Init
0000336c   Can_MainFunction_BusOff
00003274   Can_MainFunction_Mode
00003070   Can_MainFunction_Read
00002fd0   Can_MainFunction_Wakeup
00002eec   Can_MainFunction_Write
00002e34   Can_SetControllerMode
000029d4   Can_TestLoopBackModeDisable
00002964   Can_TestLoopBackModeEnable
00002758   Can_Write
000114f8   Dem_ReportErrorStatus
00011054   Det_ReportError
00012948   Device_FlashDevice
00012850   DioModuleConfiguration_0
0001282c   Dio_ChannelCheckTable
0000dea4   Dio_FlipChannel
0000de58   Dio_GetVersionInfo
0000de38   Dio_Init
00012848   Dio_PortCheckTable
0000dc50   Dio_ReadChannel
0000ddd8   Dio_ReadChannelGroup
0000db68   Dio_ReadPort
0000dd8c   Dio_WriteChannel
0000dbbc   Dio_WriteChannelGroup
0000db14   Dio_WritePort
0001293c   Dma_ChanneltoHWunit
0000fba0   Dma_DeInit
0000fb88   Dma_DisableInt
0000fb70   Dma_EnableInt
0000fb44   Dma_GetFree_Channel
08001d20   Dma_GlobalRegister
0000faac   Dma_Init
0000fa8c   Dma_IsTransferComplete
0000f738   Dma_IsrBTC
00012914   Dma_MapChannel
0000f9d0   Dma_Setup
000114e4   EcuM_CheckWakeup
000114e0   EcuM_SetWakeupEvent
000111bd   Fapi_calculateFletcherChecksum
00010ce1   Fapi_doBlankCheck
00010d75   Fapi_enableEepromBankSectors
00011321   Fapi_flushPipeline
00011495   Fapi_getNumberOfBankSectors
0000f771   Fapi_initializeFlashBanks
00010f79   Fapi_isAddressEcc
00011281   Fapi_issueAsyncCommand
000111f5   Fapi_issueAsyncCommandWithAddress
000114e8   Fapi_serviceWatchdogTimer
00010115   Fapi_setActiveFlashBank
00011225   Fapi_waitDelay
00012b04   Fee_BlockConfiguration
0000e354   Fee_Cancel
0000e2c8   Fee_EraseImmediateBlock
0000e278   Fee_GetJobResult
0000e240   Fee_GetStatus
0000e1f4   Fee_GetVersionInfo
0000e1e4   Fee_Init
0000e158   Fee_InvalidateBlock
0000e154   Fee_JobEndNotification
0000e150   Fee_JobErrorNotification
0000e140   Fee_MainFunction
0000e080   Fee_Read
0000e07c   Fee_SetMode
00012aec   Fee_VirtualSectorConfiguration
0000dfe0   Fee_Write
00012934   GptChannelConfigSet_0
00010ab8   Gpt_Ch0Isr
00010a6c   Gpt_Ch1Isr
000096bc   Gpt_CheckWakeup
08001c90   Gpt_Config_pt
000095ac   Gpt_DeInit
00008e58   Gpt_DisableNotification
00009520   Gpt_DisableWakeup
00008ef0   Gpt_EnableNotification
00009474   Gpt_EnableWakeup
00009390   Gpt_GetTimeElapsed
000092c8   Gpt_GetTimeRemaining
0000927c   Gpt_GetVersionInfo
00009120   Gpt_Init
08001ca4   Gpt_IsrIndex
000128f8   Gpt_IsrNotifyFunctions
00009068   Gpt_NotifContIsr
000090a8   Gpt_NotifSingleIsr
00009024   Gpt_SetMode
00008cb4   Gpt_StartTimer
00008af0   Gpt_StopTimer
00008ab0   Gpt_WakeupContIsr
00008a3c   Gpt_WakeupSingleIsr
0001146d   IND$CALL
00012724   IcuConfigSet_0
000071a4   Icu_CheckWakeup
00007ad8   Icu_DeInit
00007a54   Icu_DisableEdgeCount
000079d8   Icu_DisableEdgeDetection
00007974   Icu_DisableNotification
000078fc   Icu_DisableWakeup
0000719c   Icu_DoNothing
00007878   Icu_EnableEdgeCount
000077f8   Icu_EnableEdgeDetection
00007794   Icu_EnableNotification
0000771c   Icu_EnableWakeup
00007668   Icu_GetDutyCycleValues
000075cc   Icu_GetEdgeNumbers
00007554   Icu_GetInputState
000074d0   Icu_GetTimeElapsed
00007460   Icu_GetTimestampIndex
00007418   Icu_GetVersionInfo
0001114c   Icu_HetInt
00010760   Icu_Het_DeInit
000106a8   Icu_Het_Init
000072c4   Icu_Init
00007234   Icu_IrqFunction
00006fd0   Icu_ResetEdgeCount
00006ee0   Icu_SetActivationCondition
00006df4   Icu_SetMode
00006d74   Icu_StartSignalMeasurement
00006ca0   Icu_StartTimestamp
00006c20   Icu_StopSignalMeasurement
00006b90   Icu_StopTimestamp
00011110   LinIsr_0
0000c12c   Lin_AvoidCallOut
0000c060   Lin_CheckWakeup
08001fa0   Lin_FxnId
0000bf6c   Lin_GetStatus
0000bf24   Lin_GetVersionInfo
0000be3c   Lin_GoToSleep
0000ba20   Lin_GoToSleepInternal
0000bd38   Lin_Init
0000bab4   Lin_Interrupt
0000b8d0   Lin_SendFrame
0000b7c4   Lin_Wakeup
00012770   McuModuleConfiguration_0
0000c7e8   Mcu_ClearResetReason
0000c7a8   Mcu_DistributePllClock
0000c500   Mcu_GetPllStatus
0000c6b4   Mcu_GetResetRawValue
0000c6ec   Mcu_GetResetReason
0000c668   Mcu_GetVersionInfo
0000c640   Mcu_Init
0000c364   Mcu_InitClock
0000c2d4   Mcu_InitRamSection
0000c28c   Mcu_PerformReset
0000c228   Mcu_SetMode
08001870   Pdu
0000ff44   Port_GetVersionInfo
0000ff0c   Port_Init
00007ba4   Port_InitPortRegs0
0000fe88   Port_RefreshPortDirection
000127f0   Port_Runtime
0000fe50   Port_SetPinDirection
000124a4   PwmChannelConfigSet_0
0000a2cc   Pwm_DeInit
0000a114   Pwm_DisableNotification
0000a038   Pwm_EnableNotification
00009e84   Pwm_GetOutputState
00009e38   Pwm_GetVersionInfo
00009df8   Pwm_Het1EdgeNotificationISR
00010e2c   Pwm_Het1EdgeNotifyInterrupt
00009db8   Pwm_Het2EdgeNotificationISR
00010df4   Pwm_Het2EdgeNotifyInterrupt
00010638   Pwm_Het_DeInit
00010578   Pwm_Het_Init
00009d1c   Pwm_Init
0001131c   Pwm_Notification_temp
00009b90   Pwm_SetDutyCycle
000099d0   Pwm_SetOutputToIdle
000098d4   Pwm_SetPeriodAndDuty
08001fa2   Reported_Error
UNDEFED    SHT$$INIT_ARRAY$$Base
UNDEFED    SHT$$INIT_ARRAY$$Limit
00011354   SchM_Enter_Adc_ADC_EXCLUSIVE_AREA_0
00011374   SchM_Enter_Can_CAN_EXCLUSIVE_AREA_0
00011394   SchM_Enter_Dio
000113b4   SchM_Enter_Gpt_GPT_EXCLUSIVE_AREA_0
000113d4   SchM_Enter_Icu_ICU_EXCLUSIVE_AREA_0
000112d0   SchM_Enter_Mcu
000112c0   SchM_Enter_Mcu_MCU_EXCLUSIVE_AREA_0
000113f4   SchM_Enter_Port
0001130c   SchM_Enter_Pwm_PWM_EXCLUSIVE_AREA_0
00011414   SchM_Enter_Spi_SPI_EXCLUSIVE_AREA_0
00011344   SchM_Exit_Adc_ADC_EXCLUSIVE_AREA_0
00011364   SchM_Exit_Can_CAN_EXCLUSIVE_AREA_0
00011384   SchM_Exit_Dio
000113a4   SchM_Exit_Gpt_GPT_EXCLUSIVE_AREA_0
000113c4   SchM_Exit_Icu_ICU_EXCLUSIVE_AREA_0
000112bc   SchM_Exit_Mcu
000112ac   SchM_Exit_Mcu_MCU_EXCLUSIVE_AREA_0
000113e4   SchM_Exit_Port
000112fc   SchM_Exit_Pwm_PWM_EXCLUSIVE_AREA_0
00011404   SchM_Exit_Spi_SPI_EXCLUSIVE_AREA_0
080018a4   SpecialRamBlock
000126a0   SpiRuntime
08001d34   Spi_ConfigPtr_pt
0000584c   Spi_DlcBlockCbk
000057cc   Spi_DlcClose
00005780   Spi_DlcDisableInt
00005764   Spi_DlcDisableLpbk
000055e0   Spi_DlcDrive
00005590   Spi_DlcEnableInt
00005548   Spi_DlcEnableLpbk
0000531c   Spi_DlcInit
000052c0   Spi_DlcRegisterRdbk
0000523c   Spi_DlcSetEvent
08001d38   Spi_DrvStatus
00012628   Spi_HWUnit_at
000057cc   Spi_HwDeInit
0000ad60   Spi_HwInit
0000abd4   Spi_HwJobComplete
0000abd0   Spi_HwProcessState
08001c68   Spi_HwSeqEvent_at
0000aa38   Spi_HwSetEvent
00004ce8   Spi_IrqTxRx
00004550   Spi_IrqTxRxERR
0000f6fc   Spi_IrqUnit0TxRx
0000f6c0   Spi_IrqUnit0TxRxERR
0000f684   Spi_IrqUnit1TxRx
0000f648   Spi_IrqUnit1TxRxERR
0000f60c   Spi_IrqUnit2TxRx
0000f5d0   Spi_IrqUnit2TxRxERR
0000f594   Spi_IrqUnit3TxRx
0000f558   Spi_IrqUnit3TxRxERR
0000f51c   Spi_IrqUnit4TxRx
0000f4e0   Spi_IrqUnit4TxRxERR
08001c5c   Spi_JobPrioConvTbl_at
08001c60   Spi_JobsSorted_at
0001263c   Spi_RamUnit_at
00012650   Spi_UnitProperty_at
00000c14   TI_FeeInternal_AlignAddressForECC
000001f0   TI_FeeInternal_BlankCheck
000015ac   TI_FeeInternal_CheckForError
000012d8   TI_FeeInternal_CheckModuleState
00002568   TI_FeeInternal_CheckReadParameters
000001c0   TI_FeeInternal_EnableRequiredFlashSector
00001bdc   TI_FeeInternal_FeeManager
000019c4   TI_FeeInternal_FindNextVirtualSector
00000b78   TI_FeeInternal_GetArrayIndex
00000b3c   TI_FeeInternal_GetBlockIndex
00000b38   TI_FeeInternal_GetBlockNumber
00000bfc   TI_FeeInternal_GetBlockSize
000012f8   TI_FeeInternal_GetCurrentBlockAddress
00000b28   TI_FeeInternal_GetDataSetIndex
0000158c   TI_FeeInternal_GetNextFlashAddress
000014cc   TI_FeeInternal_GetVirtualSectorIndex
00000128   TI_FeeInternal_GetVirtualSectorParameter
000013a0   TI_FeeInternal_InvalidateErase
00000020   TI_FeeInternal_PollFlashStatus
00001254   TI_FeeInternal_SanityCheck
00001214   TI_FeeInternal_SetClearCopyBlockState
000011b4   TI_FeeInternal_StartProgramBlock
00000c40   TI_FeeInternal_UpdateBlockOffsetArray
00000a64   TI_FeeInternal_WriteBlockHeader
00000458   TI_FeeInternal_WriteDataF021
000009c0   TI_FeeInternal_WriteInitialize
0000088c   TI_FeeInternal_WritePreviousBlockHeader
00000668   TI_FeeInternal_WriteVirtualSectorHeader
00012154   TI_Fee_Cancel
00011d88   TI_Fee_EraseImmediateBlock
000006b8   TI_Fee_ErrorRecovery
08001d5a   TI_Fee_FapiInitCalled
000000fc   TI_Fee_GetStatus
08001d68   TI_Fee_GlobalVariables
0000ae34   TI_Fee_Init
00011f8c   TI_Fee_InvalidateBlock
0000c824   TI_Fee_MainFunction
000119ec   TI_Fee_Read
00000044   TI_Fee_SuspendResumeErase
00011518   TI_Fee_WriteAsync
08001d59   TI_Fee_bEraseSuspended
08001d5c   TI_Fee_oStatusWord
08001d64   TI_Fee_u32ActCpyVS
08001d60   TI_Fee_u32BlockEraseCount
08001d58   TI_Fee_u8DataSets
08001d44   TI_Fee_u8DeviceIndex
08001d45   TI_Fee_u8ErrEraseVS
08001d48   TI_FlashStatusWord
08001858   TestState
00011184   WdgIsr_0
0000fd74   Wdg_GetVersionInfo
0000fcfc   Wdg_Init
0000fc94   Wdg_SetMode
0000fc70   Wdg_SetTriggerCondition
08001d00   Wdg_Status
0000fbdc   Wdg_Trigger
00011011   _Fapi_EnableSectors
000114d3   _Fapi_checkWdService
000110d5   _Fapi_issueFsmCommand
00010ec5   _Fapi_loopRegionForValue
00011255   _Fapi_readDword
00012d00   __TI_CINIT_Base
00012d18   __TI_CINIT_Limit
00012cdc   __TI_Handler_Table_Base
00012ce8   __TI_Handler_Table_Limit
0000eeb0   __TI_PINIT_Base
0000eeb4   __TI_PINIT_Limit
00010c49   __TI_auto_init
000114c5   __TI_decompress_none
000114f1   __TI_decompress_rle24
00000000   __TI_static_base__
00011481   __TI_zero_init
00010bad   __aeabi_memcpy
00010bad   __aeabi_memcpy4
00010bad   __aeabi_memcpy8
00010f24   __aeabi_uidivmod
ffffffff   __binit__
ffffffff   __c_args__
00010854   _c_int00
08001d2c   _cleanup_ptr
0000edc8   _coreClearAuxiliaryDataFault_
0000eddc   _coreClearAuxiliaryInstructionFault_
0000eda0   _coreClearDataFaultAddress_
0000ed78   _coreClearDataFault_
0000edb4   _coreClearInstructionFaultAddress_
0000ed8c   _coreClearInstructionFault_
0000ed0c   _coreDisableEventBusExport_
0000ed50   _coreDisableFlashEcc_
0000ed2c   _coreDisableRamEcc_
0000ecfc   _coreEnableEventBusExport_
0000ed3c   _coreEnableFlashEcc_
0000ed60   _coreEnableIrqVicOffset_
0000ed1c   _coreEnableRamEcc_
0000ece4   _coreEnableVfp_
0000edc0   _coreGetAuxiliaryDataFault_
0000edd4   _coreGetAuxiliaryInstructionFault_
0000ed98   _coreGetDataFaultAddress_
0000ed70   _coreGetDataFault_
0000edac   _coreGetInstructionFaultAddress_
0000ed84   _coreGetInstructionFault_
0000eb6c   _coreInitRegisters_
0000ec78   _coreInitStackPointer_
0000edf0   _disable_FIQ_interrupt_
0000edf8   _disable_IRQ_interrupt_
0000ede8   _disable_interrupt_
08001d30   _dtors_ptr
0000ee00   _enable_interrupt_
0000ee90   _errata_CORTEXR4_57_
0000eea0   _errata_CORTEXR4_66_
0000ee08   _esmCcmErrorsClear_
0000ecc4   _getCPSRValue_
0000eccc   _gotoCPUIdle_
08001d24   _lock
00011467   _nop
0001145f   _register_lock
00011459   _register_unlock
000114a5   _scaleEEFclk
000114b5   _scaleMainFclk
08001d28   _unlock
00011099   abort
08001d0c   bCanBusOff
ffffffff   binit
08001514   canBaud
08001fa8   canInterruptCounter
0800150a   canTxRxPduId
08001501   canTxRxStatus
08001503   can_State
00010fc9   copy_in
0000f49c   delay
00011454   dmaGroupANotification
0000f174   esmActivateNormalOperation
0000f158   esmClearStatus
0000f14c   esmClearStatusBuffer
0000f134   esmDisableError
0000f11c   esmDisableInterrupt
0000f104   esmEnableError
0000f0ec   esmEnableInterrupt
0000f0a8   esmEnterSelfTest
0000f09c   esmError
0000f024   esmGetConfigValue
0000eff0   esmGetStatus
0000efd8   esmGetStatusBuffer
00011450   esmGroup1Notification
0001144c   esmGroup2Notification
00010790   esmHighInterrupt
0000ef50   esmInit
0000ef24   esmSelfTestStatus
0000ef14   esmSetCounterPreloadValue
0000eec8   esmSetInterruptLevel
0000eeb8   esmTriggerErrorPinReset
000110a1   exit
00010915   floor
0000f470   gpt_notification_fn
0000f1dc   main
0000d698   mapClocks
00010bad   memcpy
000112d4   memoryInit
00011448   memoryPort0TestFailNotification
00011444   memoryPort1TestFailNotification
0000e544   muxInit
0000d62c   periphInit
000114fc   phantomInterrupt
0000e3b4   pinmuxGetConfigValue
08001908   read_data
00000000   resetEntry
0000eb40   sciDisableLoopback
0000eb04   sciDisableNotification
0000eaec   sciEnableLoopback
0000eab8   sciEnableNotification
0000eaa8   sciEnterResetState
0000ea98   sciExitResetState
000103e8   sciHighLevelInterrupt
0000ea18   sciInit
0000ea0c   sciIsIdleDetected
0000ea00   sciIsRxReady
0000e9f4   sciIsTxReady
00011440   sciNotification
0000e994   sciReceive
0000e97c   sciReceiveByte
0000e964   sciRxError
0000e8d8   sciSend
0000e8c4   sciSendByte
0000e86c   sciSetBaudrate
0000e864   sciSetFunctional
0000e7b4   scilinGetConfigValue
0000d668   setupFlash
0000d5f0   setupPLL
0000d96c   sramGetConfigValue
0000d770   systemGetConfigValue
0000d728   systemInit
0000d5d4   systemPowerDown
0000d4fc   tcmflashGetConfigValue
0000d4d0   trimLPO
0000d354   vimChannelMap
0000d2fc   vimDisableInterrupt
0000d240   vimEnableInterrupt
0000cf04   vimGetConfigValue
0000cea0   vimInit
00010290   vimParityErrorHandler


GLOBAL SYMBOLS: SORTED BY Symbol Address 

address    name
--------   ----
00000000   __TI_static_base__
00000000   resetEntry
00000020   TI_FeeInternal_PollFlashStatus
00000044   TI_Fee_SuspendResumeErase
000000fc   TI_Fee_GetStatus
00000128   TI_FeeInternal_GetVirtualSectorParameter
000001c0   TI_FeeInternal_EnableRequiredFlashSector
000001f0   TI_FeeInternal_BlankCheck
00000458   TI_FeeInternal_WriteDataF021
00000668   TI_FeeInternal_WriteVirtualSectorHeader
000006b8   TI_Fee_ErrorRecovery
0000088c   TI_FeeInternal_WritePreviousBlockHeader
000009c0   TI_FeeInternal_WriteInitialize
00000a64   TI_FeeInternal_WriteBlockHeader
00000b28   TI_FeeInternal_GetDataSetIndex
00000b38   TI_FeeInternal_GetBlockNumber
00000b3c   TI_FeeInternal_GetBlockIndex
00000b78   TI_FeeInternal_GetArrayIndex
00000bfc   TI_FeeInternal_GetBlockSize
00000c14   TI_FeeInternal_AlignAddressForECC
00000c40   TI_FeeInternal_UpdateBlockOffsetArray
000011b4   TI_FeeInternal_StartProgramBlock
00001214   TI_FeeInternal_SetClearCopyBlockState
00001254   TI_FeeInternal_SanityCheck
000012d8   TI_FeeInternal_CheckModuleState
000012f8   TI_FeeInternal_GetCurrentBlockAddress
000013a0   TI_FeeInternal_InvalidateErase
000014cc   TI_FeeInternal_GetVirtualSectorIndex
0000158c   TI_FeeInternal_GetNextFlashAddress
000015ac   TI_FeeInternal_CheckForError
000019c4   TI_FeeInternal_FindNextVirtualSector
00001bdc   TI_FeeInternal_FeeManager
00002568   TI_FeeInternal_CheckReadParameters
00002758   Can_Write
00002964   Can_TestLoopBackModeEnable
000029d4   Can_TestLoopBackModeDisable
00002e34   Can_SetControllerMode
00002eec   Can_MainFunction_Write
00002fd0   Can_MainFunction_Wakeup
00003070   Can_MainFunction_Read
00003274   Can_MainFunction_Mode
0000336c   Can_MainFunction_BusOff
0000384c   Can_Init
00003910   Can_GetVersionInfo
000039d4   Can_EnableControllerInterrupts
00003ad0   Can_DisableControllerInterrupts
00003b7c   Can_ConfigRegReadBack
00003c54   Can_CheckWakeup
00003d10   Can_CheckBaudrate
00003e2c   Can_ChangeBaudrate
00004100   Can_2_Int0ISR_Fun
0000422c   Can_1_Int0ISR_Fun
00004354   Can_0_Int0ISR_Fun
00004550   Spi_IrqTxRxERR
00004ce8   Spi_IrqTxRx
0000523c   Spi_DlcSetEvent
000052c0   Spi_DlcRegisterRdbk
0000531c   Spi_DlcInit
00005548   Spi_DlcEnableLpbk
00005590   Spi_DlcEnableInt
000055e0   Spi_DlcDrive
00005764   Spi_DlcDisableLpbk
00005780   Spi_DlcDisableInt
000057cc   Spi_DlcClose
000057cc   Spi_HwDeInit
0000584c   Spi_DlcBlockCbk
0000597c   Adc_StopGroupConversion
00005a70   Adc_StartGroupConversion
00005d18   Adc_SetupResultBuffer
00005d84   Adc_ReadGroup
00005f74   Adc_ProcessConversionSingle
00005fa0   Adc_ProcessConversionLinear
00006000   Adc_ProcessConversionCircular
0000603c   Adc_ProcessBufferSingle
000060ac   Adc_ProcessBufferLinear
00006160   Adc_ProcessBufferCircular
00006214   Adc_IrqFunction
0000627c   Adc_Init
00006428   Adc_GetVersionInfo
00006474   Adc_GetStreamLastPointer
00006664   Adc_GetGroupStatus
000067a0   Adc_EnableGroupNotification
000068d8   Adc_DisableGroupNotification
00006998   Adc_DeInit
00006b88   Adc_AvoidNotification
00006b90   Icu_StopTimestamp
00006c20   Icu_StopSignalMeasurement
00006ca0   Icu_StartTimestamp
00006d74   Icu_StartSignalMeasurement
00006df4   Icu_SetMode
00006ee0   Icu_SetActivationCondition
00006fd0   Icu_ResetEdgeCount
0000719c   Icu_DoNothing
000071a4   Icu_CheckWakeup
00007234   Icu_IrqFunction
000072c4   Icu_Init
00007418   Icu_GetVersionInfo
00007460   Icu_GetTimestampIndex
000074d0   Icu_GetTimeElapsed
00007554   Icu_GetInputState
000075cc   Icu_GetEdgeNumbers
00007668   Icu_GetDutyCycleValues
0000771c   Icu_EnableWakeup
00007794   Icu_EnableNotification
000077f8   Icu_EnableEdgeDetection
00007878   Icu_EnableEdgeCount
000078fc   Icu_DisableWakeup
00007974   Icu_DisableNotification
000079d8   Icu_DisableEdgeDetection
00007a54   Icu_DisableEdgeCount
00007ad8   Icu_DeInit
00007ba4   Port_InitPortRegs0
00008a3c   Gpt_WakeupSingleIsr
00008ab0   Gpt_WakeupContIsr
00008af0   Gpt_StopTimer
00008cb4   Gpt_StartTimer
00008e58   Gpt_DisableNotification
00008ef0   Gpt_EnableNotification
00009024   Gpt_SetMode
00009068   Gpt_NotifContIsr
000090a8   Gpt_NotifSingleIsr
00009120   Gpt_Init
0000927c   Gpt_GetVersionInfo
000092c8   Gpt_GetTimeRemaining
00009390   Gpt_GetTimeElapsed
00009474   Gpt_EnableWakeup
00009520   Gpt_DisableWakeup
000095ac   Gpt_DeInit
000096bc   Gpt_CheckWakeup
000098d4   Pwm_SetPeriodAndDuty
000099d0   Pwm_SetOutputToIdle
00009b90   Pwm_SetDutyCycle
00009d1c   Pwm_Init
00009db8   Pwm_Het2EdgeNotificationISR
00009df8   Pwm_Het1EdgeNotificationISR
00009e38   Pwm_GetVersionInfo
00009e84   Pwm_GetOutputState
0000a038   Pwm_EnableNotification
0000a114   Pwm_DisableNotification
0000a2cc   Pwm_DeInit
0000aa38   Spi_HwSetEvent
0000abd0   Spi_HwProcessState
0000abd4   Spi_HwJobComplete
0000ad60   Spi_HwInit
0000ae34   TI_Fee_Init
0000b7c4   Lin_Wakeup
0000b8d0   Lin_SendFrame
0000ba20   Lin_GoToSleepInternal
0000bab4   Lin_Interrupt
0000bd38   Lin_Init
0000be3c   Lin_GoToSleep
0000bf24   Lin_GetVersionInfo
0000bf6c   Lin_GetStatus
0000c060   Lin_CheckWakeup
0000c12c   Lin_AvoidCallOut
0000c228   Mcu_SetMode
0000c28c   Mcu_PerformReset
0000c2d4   Mcu_InitRamSection
0000c364   Mcu_InitClock
0000c500   Mcu_GetPllStatus
0000c640   Mcu_Init
0000c668   Mcu_GetVersionInfo
0000c6b4   Mcu_GetResetRawValue
0000c6ec   Mcu_GetResetReason
0000c7a8   Mcu_DistributePllClock
0000c7e8   Mcu_ClearResetReason
0000c824   TI_Fee_MainFunction
0000cea0   vimInit
0000cf04   vimGetConfigValue
0000d240   vimEnableInterrupt
0000d2fc   vimDisableInterrupt
0000d354   vimChannelMap
0000d4d0   trimLPO
0000d4fc   tcmflashGetConfigValue
0000d5d4   systemPowerDown
0000d5f0   setupPLL
0000d62c   periphInit
0000d668   setupFlash
0000d698   mapClocks
0000d728   systemInit
0000d770   systemGetConfigValue
0000d96c   sramGetConfigValue
0000db14   Dio_WritePort
0000db68   Dio_ReadPort
0000dbbc   Dio_WriteChannelGroup
0000dc50   Dio_ReadChannel
0000dd8c   Dio_WriteChannel
0000ddd8   Dio_ReadChannelGroup
0000de38   Dio_Init
0000de58   Dio_GetVersionInfo
0000dea4   Dio_FlipChannel
0000dfe0   Fee_Write
0000e07c   Fee_SetMode
0000e080   Fee_Read
0000e140   Fee_MainFunction
0000e150   Fee_JobErrorNotification
0000e154   Fee_JobEndNotification
0000e158   Fee_InvalidateBlock
0000e1e4   Fee_Init
0000e1f4   Fee_GetVersionInfo
0000e240   Fee_GetStatus
0000e278   Fee_GetJobResult
0000e2c8   Fee_EraseImmediateBlock
0000e354   Fee_Cancel
0000e3b4   pinmuxGetConfigValue
0000e544   muxInit
0000e7b4   scilinGetConfigValue
0000e864   sciSetFunctional
0000e86c   sciSetBaudrate
0000e8c4   sciSendByte
0000e8d8   sciSend
0000e964   sciRxError
0000e97c   sciReceiveByte
0000e994   sciReceive
0000e9f4   sciIsTxReady
0000ea00   sciIsRxReady
0000ea0c   sciIsIdleDetected
0000ea18   sciInit
0000ea98   sciExitResetState
0000eaa8   sciEnterResetState
0000eab8   sciEnableNotification
0000eaec   sciEnableLoopback
0000eb04   sciDisableNotification
0000eb40   sciDisableLoopback
0000eb6c   _coreInitRegisters_
0000ec78   _coreInitStackPointer_
0000ecc4   _getCPSRValue_
0000eccc   _gotoCPUIdle_
0000ece4   _coreEnableVfp_
0000ecfc   _coreEnableEventBusExport_
0000ed0c   _coreDisableEventBusExport_
0000ed1c   _coreEnableRamEcc_
0000ed2c   _coreDisableRamEcc_
0000ed3c   _coreEnableFlashEcc_
0000ed50   _coreDisableFlashEcc_
0000ed60   _coreEnableIrqVicOffset_
0000ed70   _coreGetDataFault_
0000ed78   _coreClearDataFault_
0000ed84   _coreGetInstructionFault_
0000ed8c   _coreClearInstructionFault_
0000ed98   _coreGetDataFaultAddress_
0000eda0   _coreClearDataFaultAddress_
0000edac   _coreGetInstructionFaultAddress_
0000edb4   _coreClearInstructionFaultAddress_
0000edc0   _coreGetAuxiliaryDataFault_
0000edc8   _coreClearAuxiliaryDataFault_
0000edd4   _coreGetAuxiliaryInstructionFault_
0000eddc   _coreClearAuxiliaryInstructionFault_
0000ede8   _disable_interrupt_
0000edf0   _disable_FIQ_interrupt_
0000edf8   _disable_IRQ_interrupt_
0000ee00   _enable_interrupt_
0000ee08   _esmCcmErrorsClear_
0000ee90   _errata_CORTEXR4_57_
0000eea0   _errata_CORTEXR4_66_
0000eeb0   __TI_PINIT_Base
0000eeb4   __TI_PINIT_Limit
0000eeb8   esmTriggerErrorPinReset
0000eec8   esmSetInterruptLevel
0000ef14   esmSetCounterPreloadValue
0000ef24   esmSelfTestStatus
0000ef50   esmInit
0000efd8   esmGetStatusBuffer
0000eff0   esmGetStatus
0000f024   esmGetConfigValue
0000f09c   esmError
0000f0a8   esmEnterSelfTest
0000f0ec   esmEnableInterrupt
0000f104   esmEnableError
0000f11c   esmDisableInterrupt
0000f134   esmDisableError
0000f14c   esmClearStatusBuffer
0000f158   esmClearStatus
0000f174   esmActivateNormalOperation
0000f1dc   main
0000f470   gpt_notification_fn
0000f49c   delay
0000f4e0   Spi_IrqUnit4TxRxERR
0000f51c   Spi_IrqUnit4TxRx
0000f558   Spi_IrqUnit3TxRxERR
0000f594   Spi_IrqUnit3TxRx
0000f5d0   Spi_IrqUnit2TxRxERR
0000f60c   Spi_IrqUnit2TxRx
0000f648   Spi_IrqUnit1TxRxERR
0000f684   Spi_IrqUnit1TxRx
0000f6c0   Spi_IrqUnit0TxRxERR
0000f6fc   Spi_IrqUnit0TxRx
0000f738   Dma_IsrBTC
0000f771   Fapi_initializeFlashBanks
0000f9d0   Dma_Setup
0000fa8c   Dma_IsTransferComplete
0000faac   Dma_Init
0000fb44   Dma_GetFree_Channel
0000fb70   Dma_EnableInt
0000fb88   Dma_DisableInt
0000fba0   Dma_DeInit
0000fbdc   Wdg_Trigger
0000fc70   Wdg_SetTriggerCondition
0000fc94   Wdg_SetMode
0000fcfc   Wdg_Init
0000fd74   Wdg_GetVersionInfo
0000fe50   Port_SetPinDirection
0000fe88   Port_RefreshPortDirection
0000ff0c   Port_Init
0000ff44   Port_GetVersionInfo
0000ff94   Adc_IsrUnit1G2
0000ffd4   Adc_IsrUnit1G1
00010014   Adc_IsrUnit1Ev
00010054   Adc_IsrUnit0G2
00010094   Adc_IsrUnit0G1
000100d4   Adc_IsrUnit0Ev
00010115   Fapi_setActiveFlashBank
00010290   vimParityErrorHandler
000103e8   sciHighLevelInterrupt
00010578   Pwm_Het_Init
00010638   Pwm_Het_DeInit
000106a8   Icu_Het_Init
00010760   Icu_Het_DeInit
00010790   esmHighInterrupt
00010854   _c_int00
00010915   floor
000109c4   Can_2_Int0ISR
000109fc   Can_1_Int0ISR
00010a34   Can_0_Int0ISR
00010a6c   Gpt_Ch1Isr
00010ab8   Gpt_Ch0Isr
00010b10   CanIf_TxConfirmation
00010b34   CanIf_RxIndication
00010b68   CanIf_ControllerModeIndication
00010b80   CanIf_ControllerBusOff
00010bad   __aeabi_memcpy
00010bad   __aeabi_memcpy4
00010bad   __aeabi_memcpy8
00010bad   memcpy
00010c49   __TI_auto_init
00010ce1   Fapi_doBlankCheck
00010d75   Fapi_enableEepromBankSectors
00010df4   Pwm_Het2EdgeNotifyInterrupt
00010e2c   Pwm_Het1EdgeNotifyInterrupt
00010ec5   _Fapi_loopRegionForValue
00010f24   __aeabi_uidivmod
00010f79   Fapi_isAddressEcc
00010fc9   copy_in
00011011   _Fapi_EnableSectors
00011054   Det_ReportError
00011095   C$$EXIT
00011099   abort
000110a1   exit
000110d5   _Fapi_issueFsmCommand
00011110   LinIsr_0
0001114c   Icu_HetInt
00011184   WdgIsr_0
000111bd   Fapi_calculateFletcherChecksum
000111f5   Fapi_issueAsyncCommandWithAddress
00011225   Fapi_waitDelay
00011255   _Fapi_readDword
00011281   Fapi_issueAsyncCommand
000112ac   SchM_Exit_Mcu_MCU_EXCLUSIVE_AREA_0
000112bc   SchM_Exit_Mcu
000112c0   SchM_Enter_Mcu_MCU_EXCLUSIVE_AREA_0
000112d0   SchM_Enter_Mcu
000112d4   memoryInit
000112fc   SchM_Exit_Pwm_PWM_EXCLUSIVE_AREA_0
0001130c   SchM_Enter_Pwm_PWM_EXCLUSIVE_AREA_0
0001131c   Pwm_Notification_temp
00011321   Fapi_flushPipeline
00011344   SchM_Exit_Adc_ADC_EXCLUSIVE_AREA_0
00011354   SchM_Enter_Adc_ADC_EXCLUSIVE_AREA_0
00011364   SchM_Exit_Can_CAN_EXCLUSIVE_AREA_0
00011374   SchM_Enter_Can_CAN_EXCLUSIVE_AREA_0
00011384   SchM_Exit_Dio
00011394   SchM_Enter_Dio
000113a4   SchM_Exit_Gpt_GPT_EXCLUSIVE_AREA_0
000113b4   SchM_Enter_Gpt_GPT_EXCLUSIVE_AREA_0
000113c4   SchM_Exit_Icu_ICU_EXCLUSIVE_AREA_0
000113d4   SchM_Enter_Icu_ICU_EXCLUSIVE_AREA_0
000113e4   SchM_Exit_Port
000113f4   SchM_Enter_Port
00011404   SchM_Exit_Spi_SPI_EXCLUSIVE_AREA_0
00011414   SchM_Enter_Spi_SPI_EXCLUSIVE_AREA_0
00011440   sciNotification
00011444   memoryPort1TestFailNotification
00011448   memoryPort0TestFailNotification
0001144c   esmGroup2Notification
00011450   esmGroup1Notification
00011454   dmaGroupANotification
00011459   _register_unlock
0001145f   _register_lock
00011467   _nop
0001146d   IND$CALL
00011481   __TI_zero_init
00011495   Fapi_getNumberOfBankSectors
000114a5   _scaleEEFclk
000114b5   _scaleMainFclk
000114c5   __TI_decompress_none
000114d3   _Fapi_checkWdService
000114e0   EcuM_SetWakeupEvent
000114e4   EcuM_CheckWakeup
000114e8   Fapi_serviceWatchdogTimer
000114f1   __TI_decompress_rle24
000114f8   Dem_ReportErrorStatus
000114fc   phantomInterrupt
00011518   TI_Fee_WriteAsync
000119ec   TI_Fee_Read
00011d88   TI_Fee_EraseImmediateBlock
00011f8c   TI_Fee_InvalidateBlock
00012154   TI_Fee_Cancel
000124a4   PwmChannelConfigSet_0
00012628   Spi_HWUnit_at
0001263c   Spi_RamUnit_at
00012650   Spi_UnitProperty_at
000126a0   SpiRuntime
00012724   IcuConfigSet_0
00012770   McuModuleConfiguration_0
000127f0   Port_Runtime
00012800   Adc_HwUnitConfigList0_at
00012820   AdcConfigSet_0
0001282c   Dio_ChannelCheckTable
00012848   Dio_PortCheckTable
00012850   DioModuleConfiguration_0
000128e8   CanConfigSet_0
000128f8   Gpt_IsrNotifyFunctions
00012914   Dma_MapChannel
00012934   GptChannelConfigSet_0
0001293c   Dma_ChanneltoHWunit
00012948   Device_FlashDevice
00012aec   Fee_VirtualSectorConfiguration
00012b04   Fee_BlockConfiguration
00012cdc   __TI_Handler_Table_Base
00012ce8   __TI_Handler_Table_Limit
00012d00   __TI_CINIT_Base
00012d18   __TI_CINIT_Limit
08001501   canTxRxStatus
08001503   can_State
08001506   CanBusOffRecoveryStatus
0800150a   canTxRxPduId
08001514   canBaud
0800151a   CanSduPtr
0800153c   Can_CanConfig
08001558   CanMbMapping
080016d8   CanHtrhMbMapping
08001858   TestState
0800185c   CAN_RX_Int_Flag
08001860   CAN_RX_Done_Flag
08001864   CAN_TX_Done_Flag
08001868   CanRxData
08001870   Pdu
0800187c   Adc_result_buffer
080018a4   SpecialRamBlock
08001908   read_data
08001b68   CanConfigSet_0_CanController_0_CanFilterMask_0
08001b6c   CanConfigSet_0_CanController_1_CanFilterMask_0
08001b70   CanConfigSet_0_CanController_2_CanFilterMask_0
08001b74   CanConfigSet_0_CanController_0_FilterMaskList
08001b78   CanConfigSet_0_CanController_1_FilterMaskList
08001b7c   CanConfigSet_0_CanController_2_FilterMaskList
08001b80   CanConfigSet_0_CanController_0_CanControllerBaudrateConfig_0
08001b8a   CanConfigSet_0_CanController_1_CanControllerBaudrateConfig_0
08001b94   CanConfigSet_0_CanController_2_CanControllerBaudrateConfig_0
08001ba0   CanConfigSet_0_CanController_0_BaudRateConfigList
08001ba4   CanConfigSet_0_CanController_1_BaudRateConfigList
08001ba8   CanConfigSet_0_CanController_2_BaudRateConfigList
08001bac   CanConfigSet_0_CanController_0
08001bcc   CanConfigSet_0_CanController_1
08001bec   CanConfigSet_0_CanController_2
08001c0c   CanConfigSet_0_CanController_List
08001c18   CanConfigSet_0_CanHardwareObject_0
08001c30   CanConfigSet_0_CanHardwareObject_1
08001c48   CanConfigSet_0_CanHardwareObject_List
08001c5c   Spi_JobPrioConvTbl_at
08001c60   Spi_JobsSorted_at
08001c68   Spi_HwSeqEvent_at
08001c90   Gpt_Config_pt
08001ca4   Gpt_IsrIndex
08001d00   Wdg_Status
08001d0c   bCanBusOff
08001d20   Dma_GlobalRegister
08001d24   _lock
08001d28   _unlock
08001d2c   _cleanup_ptr
08001d30   _dtors_ptr
08001d34   Spi_ConfigPtr_pt
08001d38   Spi_DrvStatus
08001d44   TI_Fee_u8DeviceIndex
08001d45   TI_Fee_u8ErrEraseVS
08001d48   TI_FlashStatusWord
08001d58   TI_Fee_u8DataSets
08001d59   TI_Fee_bEraseSuspended
08001d5a   TI_Fee_FapiInitCalled
08001d5c   TI_Fee_oStatusWord
08001d60   TI_Fee_u32BlockEraseCount
08001d64   TI_Fee_u32ActCpyVS
08001d68   TI_Fee_GlobalVariables
08001fa0   Lin_FxnId
08001fa2   Reported_Error
08001fa8   canInterruptCounter
ffffffff   __binit__
ffffffff   __c_args__
ffffffff   binit
UNDEFED    SHT$$INIT_ARRAY$$Base
UNDEFED    SHT$$INIT_ARRAY$$Limit

[501 symbols]
